:1000000012C05BC580C71895189518951895189556
:10001000B9C7D4C81895EACA19CB18951895189578
:100020001895189518958FE58DBFC8E3E0E24E2E20
:1000300084E08EBFD4E0F4E05F2EEEEFF3E0A0E6C4
:10004000B0E088278D933197E9F787E189B980E09F
:1000500080BD88E18AB984B7082E877F84BF8FE18D
:1000600081BD87E081BD7CD96624579A8E988A9895
:1000700080E08FBD85E08EBD84B7877F84BF8DE132
:1000800081BD85E081BD8BB780648BBF8BB78068F5
:100090008BBF85B78C7F826085BF85B7837F886083
:1000A00085BFA0E0B3E0E8E6F8E197DAA6E0B3E0C8
:1000B000EAE6F8E192DAACE0B3E0ECE6F8E18DDAFA
:1000C000A2E1B3E0EEE6F8E188DAA8E1B3E0E0E728
:1000D000F8E183DAAEE1B3E0E6E7F8E17EDAA4E244
:1000E000B3E0ECE7F8E179DAE0E0F1E080E680D92E
:1000F00058E0C895802D76D931965A95D1F704C02D
:100100000E11111611191610E0E2F1E088E470D911
:1001100058E0C895802D66D931965A95D1F704C01C
:10012000110E11111F111120E0E4F1E080E560D9FA
:1001300058E0C895802D56D931965A95D1F704C00C
:10014000110E111111110E20E0E6F1E088E550D9F1
:1001500058E0C895802D46D931965A95D1F704C0FC
:100160001120111111110E2078947BDB8CE040D905
:1001700081B5886081BD81E090E0A5E2B1E08D931A
:100180009C9312D20091A4010F3F09F056C0ABE23C
:10019000B1E088278C93A5E2B1E00D911C910A3063
:1001A00050E0150708F024C0A5E2B1E00D911C91C4
:1001B0004EE150E008DAABE9B1E00D931C93ABE9F6
:1001C000B1E00D911C914DE150E0041B150BABE922
:1001D000B1E00D931C93ABE9B1E0ED91FC91ABE282
:1001E000B1E092E27BE722DBA5E2B1E0F4D7D3CF26
:1001F00080E090E0A5E2B1E08D939C93EFEEFFE10B
:10020000A5E2B1E092E07BE703DB81E090E0A5E2CC
:10021000B1E08D939C93EDEEFFE1A5E2B1E092E0B9
:100220007BE7F6DA80E090E0ABE9B1E08D939C9358
:100230008091E4008B7F8093E4007ED80027A4EEB9
:10024000B0E08C9184FB0EF401E041E0041709F06A
:1002500029C08091E4008F7E8093E400A5EEB0E099
:100260003FE3EAD7A5EEB0E08C91082F0A3009F001
:1002700018C0A5EEB0E0EFDA082F41E0041BA7E2BA
:10028000B1E00C93A5EEB0E0E6DAEA2FFB2F009187
:1002900027013197E01BF0400FEFA5EEB0E0A7DAA1
:1002A000E1CF8AD20027A4EEB0E08C9186FB0EF459
:1002B00001E040E0041781E009F080E08F9300271F
:1002C000A4EEB0E08C9183FB0EF401E041E0041752
:1002D00081E009F080E09F918923882309F4D8C048
:1002E0008091E400877F8093E400BDD8A9E2B1E06B
:1002F0002C93AAE2B1E01C9300912A010F3710F071
:1003000009F001C005C0AAE2B1E08C9180588C933D
:1003100000912A01003081E008F480E08F93009181
:100320002A01093081E010F009F080E09F918923D3
:10033000882309F437C0ABE2B1E075D7EAE2F1E017
:10034000CED90027A4EEB0E08C9185FB0EF401E03D
:1003500041E0041781E009F080E08F9300912A01C9
:10036000003081E009F480E09F918923882309F41B
:1003700018C08091E4008F7D8093E400AAE2B1E090
:100380000C914EE1049F0C92AAE2B1E08C918D5148
:100390008C93AAE2B1E0EC91FF27ABE2B1E092E2EC
:1003A00053DA71C040919D01041709F007C0ABE218
:1003B000B1E039D7E8E6F8E110D965C040919E0177
:1003C000041709F007C0ABE2B1E02DD7EAE6F8E187
:1003D00004D959C040919F01041709F007C0ABE24E
:1003E000B1E021D7ECE6F8E1F8D84DC04091A0018A
:1003F000041709F007C0ABE2B1E015D7EEE6F8E16B
:10040000ECD841C04091A101041709F00BC0ABE248
:10041000B1E0E2E8F8E1E1D88091E4008062809305
:10042000E40031C04091A301041709F01DC0ABE204
:10043000B1E011DA082F013009F005C0ABE2B1E0FC
:1004400088278C9310C0ABE2B1E005DA082F41E0B9
:10045000041BA7E2B1E00C93EBE2F1E0009127016D
:10046000ABE2B1E0C4D90FC04091A201041709F07A
:100470000AC0EBE2F1E0A5EEB0E0ADD9ABE2B1E04D
:1004800088278C93C2D08091E40080688093E40038
:100490000027A4EEB0E08C9182FB0EF401E041E075
:1004A000041709F06EC081E08093A60181E080937B
:1004B000A6010091A601093010F009F054C0A6EA87
:1004C000B1E0AD90BB24AEE6B1E0AA0DBB1D0C912E
:1004D000003380E010F009F081E08F93A6EAB1E0EC
:1004E000AD90BB24AEE6B1E0AA0DBB1D0C910A3362
:1004F00081E008F080E09F918923882309F42CC0D3
:10050000A6EAB1E0AD90BB24AEE6B1E0AA0DBB1DFA
:100510008C918093A701A7EAB1E08C9180538C93D2
:10052000A7EAB1E00C914EE1049F0C92A7EAB1E07A
:100530008C918D518C93A7EAB1E0EC91FF27A6EA4C
:10054000B1E00D91112742E250E03DD8ACEAB1E0B4
:10055000A00FB11F92E278D9A6EAB1E08C918F5F2B
:100560008C9308F4A6CF8091E4008B7F8093E40005
:10057000ABE2B1E088278C938091E400806880939F
:10058000E4000027A4EEB0E08C9187FB0EF401E0BC
:1005900041E0041709F006C08091E4008F77809352
:1005A000E4003ED0A8954ACEEFEEFFE1A4EAB1E028
:1005B00091E04AD9E0EFFFE1ADE9B1E091E044D943
:1005C000E1EFFFE1AEE9B1E091E03ED9E2EFFFE11A
:1005D000AFE9B1E091E038D9E3EFFFE1A0EAB1E0A3
:1005E00091E032D9E4EFFFE1A1EAB1E091E02CD94A
:1005F000E5EFFFE1A2EAB1E091E026D9E6EFFFE105
:10060000A3EAB1E091E020D90895A5EEB0E053D679
:1006100058D608958091E40080618093E4000895A5
:10062000EBE2F1E0ADE4B1E0D6D881E08093A50142
:10063000ADE4B1E010D9482F0091A501041710F0E6
:1006400009F071C0A5EAB1E0AD90BB24ACE4B1E023
:10065000AA0DBB1D0C91013809F00BC085EFA5EA6E
:10066000B1E0AD90BB24ACE4B1E0AA0DBB1D8C930E
:1006700053C0043809F00BC081EEA5EAB1E0AD909B
:10068000BB24ACE4B1E0AA0DBB1D8C9345C004397A
:1006900009F00BC08FEEA5EAB1E0AD90BB24ACE44D
:1006A000B1E0AA0DBB1D8C9337C0013E09F00BC011
:1006B00084E0A5EAB1E0AD90BB24ACE4B1E0AA0DC2
:1006C000BB1D8C9329C00E3809F00BC081E0A5EA50
:1006D000B1E0AD90BB24ACE4B1E0AA0DBB1D8C939E
:1006E0001BC0093909F00BC082E0A5EAB1E0AD906A
:1006F000BB24ACE4B1E0AA0DBB1D8C930DC00A393C
:1007000009F00AC083E0A5EAB1E0AD90BB24ACE4F7
:10071000B1E0AA0DBB1D8C93A5EAB1E08C918F5F6F
:100720008C9308F485CF8FE711E015D6EDE4F1E066
:1007300000E1A9E7B1E05BD8A9E7B1E0EFD5E4E9D2
:10074000F8E1F2D5F7D5ADE4B1E085D8A7E2B1E0A4
:100750008C9381E1EDE4F1E000E20A93AAE8B1E0D4
:100760003FD8AAE8B1E0DAD5E4E9F8E1DDD5002721
:10077000A4EEB0E08C9181FB0EF401E041E004179F
:1007800009F019C081B5886181BD877F81BD84EF83
:1007900091E05AD681B5886081BDABE2B1E088278F
:1007A0008C938091E4008D7F8093E4008091E4003D
:1007B00080688093E4000895A5EEB0E08C91082F46
:1007C000033209F0F2C084E0E5EEF0E001E00A93C4
:1007D000AAEAB1E005D8AAEAB1E08C91A8EAB1E0B2
:1007E0008D9388278C93A8EAB1E00D911C91053276
:1007F00050E0150709F0D7C082E0E5EEF0E002E036
:100800000A93AAEAB1E0ECD7AAEAB1E0B2D7A8EA23
:10081000B1E00D931C93A8EAB1E00D911C91013059
:1008200050E0150781E008F480E08F93A8EAB1E07A
:100830000D911C91093050E0150781E010F009F08E
:1008400080E09F918923882309F447C0A8EAB1E09A
:100850000D911C914EE150E0B6D6A8EAB1E00D939F
:100860001C93A8EAB1E00D911C914DE150E0041BEE
:10087000150BA8EAB1E00D931C9385E0E5EEF0E0DE
:1008800000E20A93AAEAB1E0ABD7A8EAB1E0ED91A1
:10089000FC91AAEAB1E092E27BE7C8D7A5EEB0E00E
:1008A000E6EAF8E19AD6A5EEB0E0BDD4E8EAF1E0D8
:1008B00007D7A5EEB0E0B7D4E2EBF8E18ED6EAEACE
:1008C000F1E0A5EEB0E0AFD486D7A5EEB0E0ABD4B2
:1008D000EAEBF8E182D699DE65C0033650E01507F1
:1008E00009F002C064D05EC0023650E0150709F07E
:1008F0002EC085E0E5EEF0E005E00A93AAEAB1E05B
:100900006FD7AAEAB1E035D7A8EAB1E00D931C93FE
:10091000A8EAB1E00D911C91083E5DEF150710F0BB
:1009200009F001C006C088EE9DEFA8EAB1E08D9302
:100930009C93EDEEFFE1A8EAB1E092E07BE768D797
:10094000A5EEB0E0E8ECF8E148D65FDE2BC001365A
:1009500050E0150709F020C08091E4008460809386
:10096000E40085E0E5EEF0E009E00A93AFE6B1E0EF
:1009700037D7A5EEB0E0E6EEF8E12FD6EFE6F1E0EE
:10098000A5EEB0E050D427D7A5EEB0E04CD4E2EF0E
:10099000F8E123D63ADE06C0A5EEB0E0E0E0F9E1EA
:1009A0001CD633DE01C031DE01C02FDE089581B5D3
:1009B000886181BD877F81BD8091E40080648093E0
:1009C000E40081E080932A0300912A03083008F0B4
:1009D0005EC0B2D4EAE1F9E1A7D485EF03D5E8E23D
:1009E000F9E1A2D4A7D4AAE2B3E00D91112746E021
:1009F00050E0E9D5AAEFB2E0A00FB11F8FD4EAE230
:100A0000F9E192D485EFEED4EEE2F9E18DD42BD565
:100A1000A9E2B1E02C93AAE2B1E01C9300912A0173
:100A20000F3710F009F001C005C0AAE2B1E08C91C7
:100A300080588C9300912A010F3709F4E8CFAAE27D
:100A4000B3E00D9111274FEE5FE1040F151FABE2EC
:100A5000B3E00D931C93ABE2B3E0ED91FC91AAE2FD
:100A6000B1E091E07BE7D4D667D4A8E0B4E0EAE255
:100A7000F1E035D651D4E4E3F9E156D480ED97E0C6
:100A8000E3D4AAE2B3E08C918F5F8C939DCF54D4D2
:100A9000ECE3F9E149D44ED4EAE4F9E145D484DD4C
:100AA00080ED97E0D1D448D48091E4008F7B80938F
:100AB000E40081B5886081BD08950F921F922F9246
:100AC0003F924F925F927F92AF92BF920F931F938C
:100AD0002F933F934F935F936F937F938F939F9346
:100AE000AF93BF93CF93DF93EF93FF938FB78F9322
:100AF0002FD5ABE9B1E08D9388278C93ABE9B1E0BA
:100B00000D911C910D3050E0150709F00BC0EBE280
:100B1000F1E0A5EEB0E05FD6ABE2B1E088278C93C0
:100B200074DDC7C1083050E0150709F01DC0ABE205
:100B3000B1E091D6082F013009F005C0ABE2B1E079
:100B400088278C9310C0ABE2B1E085D6082F41E036
:100B5000041BA8E2B1E00C93EBE2F1E00091280164
:100B6000ABE2B1E044D6A5C10B3A50E0150709F05D
:100B70000CC0E1E0F0E0ABE2B1E092E265D6EBE27E
:100B8000F1E0ADE4B1E027D694C10C3A50E015078E
:100B900009F00CC0EFE1F0E0ABE2B1E092E254D634
:100BA000EBE2F1E0ADE4B1E016D683C10D3A50E0DE
:100BB000150709F00CC0EDE3F0E0ABE2B1E092E222
:100BC00043D6EBE2F1E0ADE4B1E005D672C10E3AF6
:100BD00050E0150709F00CC0EBE5F0E0ABE2B1E046
:100BE00092E232D6EBE2F1E0ADE4B1E0F4D561C1DE
:100BF0000F3A50E0150709F00CC0E9E7F0E0ABE26E
:100C0000B1E092E221D6EBE2F1E0ADE4B1E0E3D570
:100C100050C1003B50E0150709F00CC0E7E9F0E0D7
:100C2000ABE2B1E092E210D6EBE2F1E0ADE4B1E08C
:100C3000D2D53FC1013B50E0150709F00CC0E5EBF0
:100C4000F0E0ABE2B1E092E2FFD5EBE2F1E0ADE43F
:100C5000B1E0C1D52EC1023B50E0150709F00CC030
:100C6000E3EDF0E0ABE2B1E092E2EED5EBE2F1E0F1
:100C7000ADE4B1E0B0D51DC1033B50E0150709F06C
:100C80000CC0E1EFF0E0ABE2B1E092E2DDD5EBE2E7
:100C9000F1E0ADE4B1E09FD50CC1053B50E0150794
:100CA00009F00DC0E1E0F0E0ABE2B1E092E27BE7F9
:100CB000BDD58091E40084608093E400FAC0063BD7
:100CC00050E0150709F00DC0EFE1F0E0ABE2B1E054
:100CD00092E27BE7ABD58091E40084608093E400EE
:100CE000E8C0073B50E0150709F00DC0EDE3F0E068
:100CF000ABE2B1E092E27BE799D58091E4008460B9
:100D00008093E400D6C0083B50E0150709F00DC001
:100D1000EBE5F0E0ABE2B1E092E27BE787D58091D2
:100D2000E40084608093E400C4C0093B50E01507F0
:100D300009F00DC0E9E7F0E0ABE2B1E092E27BE759
:100D400075D58091E40084608093E400B2C00A3BD2
:100D500050E0150709F00DC0E7E9F0E0ABE2B1E0C3
:100D600092E27BE763D58091E40084608093E400A5
:100D7000A0C00B3B50E0150709F00DC0E5EBF0E01B
:100D8000ABE2B1E092E27BE751D58091E400846070
:100D90008093E4008EC00C3B50E0150709F00DC0B5
:100DA000E3EDF0E0ABE2B1E092E27BE73FD580918A
:100DB000E40084608093E4007CC00D3B50E01507A4
:100DC00009F00DC0E1EFF0E0ABE2B1E092E27BE7C9
:100DD0002DD58091E40084608093E4006AC00E3BCE
:100DE00050E0150709F040C0ACECB1E00D911C914A
:100DF000003050E0150709F023C0EDEEFFE1ACEC48
:100E0000B1E092E021D589B7846089BFABE2B1E05F
:100E1000E6E5F9E1E2D384E8ABE2B1E08F9303D2F7
:100E20008F918D9388278C93ABE2B1E0FCD1EEE5F6
:100E3000F9E1D3D38091E40082608093E40013C091
:100E400080E090E0ACECB1E08D939C9389B78B7F10
:100E500089BFABE2B1E0E2E6F9E1BFD38091E40003
:100E600082608093E40025C00F3B50E0150709F035
:100E70000CC08091E40084608093E400EBE2F1E038
:100E800009E0AFE6B1E0B3D414C0ABE9B1E00D9135
:100E90001C91003050E0150709F40BC0ABE9B1E03C
:100EA0008C91ABE2B1E08F93BED18F918D93882767
:100EB0008C938AB780648ABF80E090E0ABE9B1E0B0
:100EC0008D939C938091E40080688093E4008F91DF
:100ED0008FBFFF91EF91DF91CF91BF91AF919F9124
:100EE0008F917F916F915F914F913F912F911F91C2
:100EF0000F91BF90AF907F905F904F903F902F9059
:100F00001F900F9018950F921F922F923F924F9221
:100F10005F927F92AF92BF920F931F932F933F9355
:100F20004F935F936F937F938F939F93AF93BF93F1
:100F3000CF93DF93EF93FF938FB78F938091E4006C
:100F400088608093E4008AB780688ABF8F918FBFE2
:100F5000FF91EF91DF91CF91BF91AF919F918F91D1
:100F60007F916F915F914F913F912F911F910F91C1
:100F7000BF90AF907F905F904F903F902F901F90C9
:100F80000F9018950F921F922F923F924F925F925F
:100F90007F92AF92BF920F931F932F933F934F93E4
:100FA0005F936F937F938F939F93AF93BF93CF93F1
:100FB000DF93EF93FF938FB78F93ACECB1E00D917C
:100FC0001C91003050E0150709F45AC00091A701A8
:100FD000003081E009F080E08F930091A701093093
:100FE00080E010F009F081E09F91892B882309F4BB
:100FF00003C081E08093A701ACECB1E08D919C919E
:1010000090934D0080934C00A7EAB1E00D91112719
:1010100042E250E0D8D2ACEAB1E0A00FB11F8C910F
:10102000082F003081E009F080E08F930091A70144
:101030000A3081E008F080E09F918923882309F439
:1010400006C0A7EAB1E08C918F5F8C93DDCF009151
:10105000A7010A3008F014C0E7EAF1E00191112776
:1010600042E250E0B0D2ECEAF1E0E00FF11FA5EE71
:10107000B0E0B1D3CADAA7EAB1E08C918F5F8C936C
:101080008F918FBFFF91EF91DF91CF91BF91AF9182
:101090009F918F917F916F915F914F913F912F9190
:1010A0001F910F91BF90AF907F905F904F903F90B6
:1010B0002F901F900F901895F894FFCF00B300AFBA
:1010C000ADABAC0000B4B2B0AE0000000000000058
:1010D000007131040404797361773200006378642D
:1010E000653433040420766674723500006E6268DD
:1010F000677A3607082C6D6A75373800002C6B69E3
:101100006F303904042E2D6C9470E100000084E4EB
:10111000815C040404040D0404230000003C00006E
:10112000000008000031003437000000302CB135D9
:1011300036380000002B332D2A39BE0000BD00B91F
:10114000B7B5B6000000BCBAB8000000000000004F
:1011500000512100000059534157220000435844D8
:10116000450023000020564654522500004E4248B8
:10117000475A2600004C4D4A552F2800003B4B494A
:101180004F3D2900003A5F4C99503F0000008E000F
:101190009A60000000000D5E002A0000003E000082
:1011A000000800003100343700000000302CBB354F
:1011B00036380000002B332D2A39BF008F939F93C0
:1011C0008FB73395539509F443959CE892BF9F914F
:1011D0008FBF8F911895ED91FC91EF5FFF4FFC93BE
:1011E000EE93089504D0EFD100FC0CD008950024B4
:1011F000E89457FF02C009D0689400F80BD010F8AB
:101200000124089502D009D00895509540954F5F6C
:101210005F4F0895E89417FF0895009510950F5FAC
:101220001F4F689408958F938D918823E9F7119744
:101230008F910895A8E0B4E018D0883091F08D30F7
:1012400039F03323C9F38D933A9563FE3DD0F4CF43
:1012500063FC04C08DE038D08AE036D088278C93B8
:10126000089532D011973395E7CF0F929F93AF93A4
:10127000BF937F938091A1008823E1F3F89480913C
:10128000A1008A958093A10090919F00A0E6B0E014
:10129000A90F0024B01D8C9193959F3309F49927D1
:1012A00090939F0078947F91BF91AF919F910F9001
:1012B0000895A8E0B4E08D91882311F005D0FBCF0C
:1012C00008958DE001D08AE09F939FB79F93AF93DD
:1012D000BF930F937F939091E3009F33E1F3F894D2
:1012E0009091E30093959093E30099270091E20099
:1012F000A2EAB0E0A00FB91F8C9303950F3309F455
:1013000000270093E200559A7F910F91BF91AF9112
:101310009F919FBF9F910895A8E0B4E08D9188238D
:1013200011F060D0FBCF08955DD1802D11F05AD01F
:10133000FBCF089580EC5CC081E05AD00ED080E8ED
:1013400057C08FE7213039F08FEB223021F08FE842
:10135000233009F08FEC810F4BC083E0992774C0D4
:101360008AEF90E071D0A59AA49AA39AA29AB99A0A
:10137000B89AC09885E090E067D0C198AD98AC98D5
:10138000AB9AAA9AC19AEF93FF93EDE6F1E050D0A1
:10139000FF91EF91C19855D0C19AEF93FF93EDE67D
:1013A000F1E046D0FF91EF91C1984BD0C19AEF93F5
:1013B000FF93EDE6F1E03CD0FF91EF91C19841D071
:1013C000AA98C19AEF93FF93EDE6F1E031D0FF9137
:1013D000EF91C19836D088E20BD08EE009D086E03C
:1013E00007D00895C09A829505D004D02AD00895D8
:1013F000C098F9CF859510F4AA9A01C0AA9885954E
:1014000010F4AB9A01C0AB98859510F4AC9A01C06A
:10141000AC98859510F4AD9A01C0AD98C19AEF9340
:10142000FF93EDE6F1E004D0FF91EF91C1980895AC
:101430003197F1F70895689462F80895E89462F896
:10144000089581E090E000C0EF93FF93EE27E82B32
:10145000E92B31F0E6E6FEE03197F1F70197D1F79D
:10146000FF91EF9108950F933F934F935F932F92C6
:101470003F928F939F938FB78F9383B78F938260A1
:1014800083BF89B78F93816089BF8CE882BF55275E
:1014900044273327483008F047C0373324F4839B70
:1014A000F8CFF8CF41C04830ECF78399FCCF332711
:1014B0003232D4F5839BFCCF932F33271127222779
:1014C000913110F0969511E0292E2694322C290E98
:1014D000990F390E113021F0321534F58399FCCF74
:1014E00033270CE03215F0F3839909C08894111F5B
:1014F000221F3315CCF4839BFCCF332708C00894FC
:10150000111F221F331584F48399FCCF33270A95CA
:1015100049F7912F991F221F991F221F25FB17F9A9
:1015200026FB16F92F7102C01FEF2FEF8F9189BF95
:101530008F9183BF8F918FBF9F918F913F902F90FD
:101540005F914F913F910F91089562FA26F432C056
:10155000E89462F80BE08299F8CF023038F031F06D
:101560000B3008F003C0969586999068829BFECF59
:101570000A9589F7153619F4892F11270895903F98
:1015800019F4689465F816C0923111F0993529F470
:1015900065FAAEF0689464F80DC065FA6EF064FA0E
:1015A0000EF49058ECEBF0E18827E90FF81FC8958E
:1015B000802D089588270895E89465F8FBCFE89476
:1015C00064F865F8F7CF0F92B801469F8001479FF6
:1015D000100D569F100D0F90089504D00D9200200D
:1015E000E1F70895C8953196002008957F930F93F1
:1015F000AF93BF938F939F938FB78F93E89480910E
:10160000A1000FE3081B19F49CB115DF13C0009172
:10161000A000A0E6B0E077279CB1A00FB71F9C9375
:10162000689483958093A10003950F3309F40027F4
:101630000093A0009D3009F4EDD78F918FBF9F914B
:101640008F91BF91AF910F917F9118957F93AF9339
:10165000BF938F939F938FB78F939091E3009923BC
:1016600099F09A959093E3009927A2EAB0E08091CF
:10167000E100A80FB91F9C9183958F3309F4882747
:101680008093E1009CB901C055988F918FBF9F91C5
:101690008F91BF91AF917F911895040F151F261F51
:1016A000371F0895000F111F221F331F0895009543
:1016B0001095209530950F5F1F4F2F4F3F4F089586
:1016C000019110810EC001911191219130810BC0C7
:1016D0000191108117FF05C03FEF2FEF04C000817B
:1016E00011272227332737FF03C0E1DF8DE28D93D7
:1016F000CF93DF93CF92DF92EF92AA24BB24CC2426
:10170000DD24EE2440E2CAE0DD2755E093E3888142
:10171000890F87FD9F7083FD907F891B89935A9560
:10172000A9F7C0DFAA1CBB1CCC1CDD1CEE1C4A9513
:1017300051F7E894EFE0FF2782910ED0EB30E0F70D
:101740001EF068948A2D0CD088278D93EF90DF903F
:10175000CF90DF91CF910895982F829501D0892F56
:101760008F70805D26F0803309F4089568948D931E
:10177000089500271127222733271DD08A3328F404
:10178000803318F005D015D0F9CF0EF490CF08951E
:1017900080538F93402F512F622F732F83DF82DF6F
:1017A0007CDF80DF8F919927080F191F291F391FB0
:1017B00008958D910895E894FCDF8032E9F38B322F
:1017C000D9F38930C9F38D3211F46894F2CF0895BA
:1017D00088278D93089581918D938823E1F708954B
:1017E00009919191992351F08A95D9F73197819177
:1017F0008D930A9519F08823D1F70895E9CFE199DF
:10180000FECFEEBBFFBB3196089591E001C092E0A0
:101810007B3751F47FB7F894F2DF8D918DBBE29A5C
:10182000E19A9A95C9F77FBF77270895E8DF8D91F0
:101830007B3729F48DBBE29AE19A8823B9F77727A1
:10184000089591E001C092E0DADFE09A8DB38D93C4
:101850009A95D1F708958FEF83959D919923E1F79C
:101860000895689463F8089521003F003A003D0010
:1018700053746F726500456E746572004261636BEC
:10188000000053706569636865726E756D6D657291
:101890003A2000002020202020202020202020206E
:1018A0002020202000002353706569636865722042
:1018B000000020576572742000002067657363681C
:1018C00072696562656E00002320476573636877FF
:1018D000696E6469676B65697420676573706569B3
:1018E00063686572740023204162666F6C67653AB5
:1018F0002000206765737065696368657274000015
:10190000232053706569636865726572726F722017
:1019100046422D4D6F64756C0000426974746520F9
:101920005461737465206600720020647200636BFA
:10193000656E00002053746F726564004642206536
:10194000696E6C65726E656E000069737420626505
:10195000656E6465740054696D6572206C0075660F
:10196000740054696D657220697374206175730029
:00000001FF
